:10000000660A2A00EA02020A0008E20114081B0834
:10001000170813081A0816081208190815081108F5
:10002000180810080008000800080008740C2A00CE
:100030000605EA02190A060400082C0016090C0C31
:100040005D09020C2700050C2B000C022D0016097F
:100050005C098D065A096D03EB02270A16090C0C80
:100060005D09E702230A3D0C5D0900080E0C010939
:100070006606580A080C2B006C0000000000000007
:100080000000000003041D0C01092C0366074B0A45
:10009000EC0500004E0A000000000000EB02410ADF
:1000A00000001E0C01096607580A0304040000083A
:1000B0000305FF08020C5D0A040C2900AF0C2800A0
:1000C000E802600A0400E9025E0A0008800C0200EF
:1000D0000E0C060006046E006F00700071007200C6
:1000E00004006606700A36090306700A0C020D0F3A
:1000F0004306860A0F022E0010022F001102300064
:10010000120231000C020F0E3200700A180C1D0989
:100110000E0205091D090F0205091D091002050936
:100120001D09110205091D09120205091D096B0AA5
:080800000F00020002000500D8
:021FFE00ED0FE5
:00000001FF
